:10000000A00168299000240884002208E0208413BD
:100010000005181C2206031920281008031D1828A3
:100020001608FF3E031C21280A30F5201608212857
:10003000100AFF3003192028100B20281708212848
:1000400099090310191803146329A016A01EA01201
:1000500020192E28A100201503106329201A362804
:10006000920020164D2003183B2812085420031834
:100070003B28A01E632946206B2020112012A011CE
:10008000240884002208841780044C282408840053
:100090002209800584178005080040206B20462037
:1000A00067202108A01901388E0008308F008E0DBE
:1000B00003184020031C46206B2067208F0B572815
:1000C00040206B202408840022080005FF3E2508FC
:1000D0008400230949282508840023088004841704
:1000E000230980054C2891019000A11727308F002B
:1000F0001030862003308F00E83086208F01643076
:1001000086208F010A308620100891288E00110861
:100110008D0010088C0031210C08031DA113A11BB8
:100120000800303EA018BD28930086118316861162
:1001300083123A308D009830032186108316861082
:1001400083123330920083160F3086058312D1203C
:100150000F308D00DC300321D1203C300221D12032
:1001600022309200D1202030BC200C30BC20063040
:10017000BC20A0141308BD2820149200201CCB28FA
:100180008610033C031CD028D0203E308D008030E8
:100190000321031408002014FE3C0319632986146C
:1001A000201C20100F3086051208F03986048615B1
:1001B000920E86112018D12828300221031408003D
:1001C00084178004632989008316081483120808A1
:1001D000632988008316081555308900AA308900E4
:1001E00088148818F128081163298F018E00FF30C8
:1001F0008E07031C8F07031C632903308D00DF303B
:100200000321F7288D01E83E8C008D09FC30031C8A
:100210000C298C07031809298C0764008D0F092904
:100220000C1812298C1C16290000162908008E00B3
:10023000023021298E00063021298F018E000430E2
:10024000212994000F080D02031D28290E080C0215
:10025000043003180130031902301405031DFF3068
:10026000632910309200910190010D0D900D910DB8
:100270000E0890020F08031C0F0F91020318472964
:100280000E0890070F0803180F0F910703108C0D2D
:100290008D0D920B35290C086329103094008D01C7
:1002A0008C01930C920C031C5B290E088C070F0821
:1002B00003180F0F8D078D0C8C0C910C900C940B68
:1002C0005129100863298313031383126400080063
:1002D000831605148514051505168312C230B20065
:1002E000C030AE004430AF000130B7006430F520BC
:1002F000061183160611FE308312922001309220DF
:100300005430922058309220203092204130922058
:100310005430922056309220203092203230922059
:100320002E30922033309220473092204830922055
:100330007A309220203092207630922037309220EE
:1003400003308F00E830F6200030E320B0000130A9
:10035000E320B1002E083007AC002F080318013E3F
:100360003107AD000630A4000130A2000630A50020
:100370000230A300320827202D0827202C08272030
:100380008E3025204622712201308F00F430F62075
:100390000530A4000130A20098010A309600023016
:1003A00097000130990033080220B3000318092A8E
:1003B0000530A4000230A20098010A3096000230F5
:1003C00097000130990034080220B40003181A2A5B
:1003D0000530A4000430A2009801FF309600970178
:1003E0000130990036080220B6000318B92A0530FA
:1003F000A4001030A2009801FF3096009701013050
:10040000990035080220B5000318382A6430F52019
:10041000C8293708B0070318B10A30088C00310822
:100420008D000E308F0010301A21031D192AB001E3
:10043000B101AA2930088C0031088D0037081D2130
:10044000031D352A30088C0031088D008F010030E3
:100450001721031D302A3708B002031CB103AA2953
:100460001030B0000E30B100AA29B001B101AA29A4
:1004700064003708083C0319422A0310B70D8C2288
:100480007122C8290130B7008C22C82980302C0283
:10049000A6003E30031C013E2D02A70026088C005A
:1004A00027088D0008308E008F013121A8000D082B
:1004B000A90026088C0027088D0008308E008F01C7
:1004C000312110089E0011089F007D309200930199
:1004D0001E088E001F088F004D21AA001108AB00D6
:1004E0000800FE309220013092200230732029084B
:1004F0009100280874202E3092202B0891002A08A1
:100500007420203092204D309220483092207A3052
:100510009220203092200800FE309220013092205C
:1005200050309220613092207330922020309220FF
:100530006430922065309220203092207D309200ED
:10054000930137088E008F014D219E0011089F00F6
:100550001F0891001E087420203092206B309220DA
:10056000483092207A30922003308F00E830F62015
:10057000080089013008E920013089003108E920AC
:02058000C82988
:02400E00F53F7C
:04420000C0000300F7
:00000001FF
